:1000000052C2000088C2000086C2000084C2000004
:1000100082C2000080C200007EC200007CC20000DC
:100020007AC2000078C200000C940B2D0C94F02DC5
:100030000C94960F70C200006EC200006CC20000EB
:100040006AC2000068C2000066C2000064C200000C
:1000500062C200000C94E72C5EC200005CC200008B
:100060005AC2000058C2000056C2000054C200002C
:1000700052C2000050C200004EC200004CC200003C
:100080004AC2000048C2000046C2000044C200004C
:1000900042C2000040C200003EC200003CC200005C
:1000A0003AC2000038C2000036C200000501090251
:1000B000A10185020901A1000509190129081500FE
:1000C0002501950875018102050109300931158165
:1000D000257F95027508810609381581257F9501D0
:1000E00075088106050C0A38021581257F95017572
:1000F000088106C0C005010980A101850319012AF4
:10010000B700150126B700950175108100C0050CD8
:100110000901A101850419012AA002150126A002E6
:10012000950175108100C00660FF0961A101096297
:10013000150026FF00952075088102096315002629
:10014000FF00952075089102C005010906A101056F
:100150000719E029E7150025019508750181029529
:1001600001750881010507190029FF150026FF0008
:100170009506750881000508190129051500250156
:10018000950575019102950175039101C00000006C
:10019000000000000000000000000000000000005F
:1001A000000000000000000000000000000000004F
:1001B000007E0F00D4FFFFFFC700000078000000A2
:1001C00000000000002A2B280000000000000000B2
:1001D000000000000000000029000000002C1E3478
:1001E00020212224342627252E362D3738271E1F7E
:1001F000202122232425263333362E37381F0405A9
:10020000060708090A0B0C0D0E0F10111213141516
:10021000161718191A1B1C1D2F3130232D350405F4
:10022000060708090A0B0C0D0E0F101112131415F6
:10023000161718191A1B1C1D2F3130354C09025B7B
:1002400000030100A03209040000010301010009BC
:100250002111010001224400070581030800010962
:100260000401000203000000092111010001222203
:100270000007058203200001070503032000010990
:100280000402000103000000092111010001227B8A
:10029000000705840320000112010002000000088D
:1002A00043506F4D0100010203011C0376006900F9
:1002B00061006C003A0066003600340063003200D2
:1002C00062003300630000000C034D006F007500F6
:1002D0007300650000000E0350006C006F006F009B
:1002E00070007900000004030904D100D300D2009B
:1002F000D400D50019010601007EFD377A585A0056
:100300000004E6D6B4460200210116000000742F56
:10031000E5A3E00205013A5D003D8889C65436C375
:10032000174FE4E468771740EC062B597485A6E56F
:1003300090A005239DD3264B55FC9FAFBED5FF044F
:10034000EDF4BE5333864EB7E68EA21BC05FE64C7B
:100350004A71611FC39F96FA33DC2E9DD4F4EFF8E7
:1003600096A1E2BE82C0E5B408712BC8E1FCB51EBF
:10037000D59D49CC0C964E64593FF7879DA63E19F2
:10038000DF63FB7CF6CCBBF3508A5D447E2915EC21
:10039000103DD179C80F70FC6CC8E43BAD9A221EA9
:1003A000C3AB155D85667ADA9856B6430FB6E72378
:1003B000436AFD7D2D71CDAB28CE551136C97D86A2
:1003C000CBD01C3BEEBAD40D475924B7DE294C7470
:1003D00065545D59D0275280446AB2BD35A2EB64A2
:1003E000D53D28796318FA1797AE585E5E8FA51F22
:1003F000CEB8FF61D93587350E84DDF005B1071F12
:100400007E6B66D7A44F8444D6603475D939F963BE
:1004100064F089D48ECF4AA39525E49A155B161D06
:10042000589F5D442B7FDC5C73E86A456A84003426
:100430006152070EB192C9D0BD9CF5837580159F9E
:1004400040E65E4825741983D240E8552FF03163A9
:10045000F89B00000000424E777FBEA00C4D0001CB
:10046000D60286040000B439C9B2B1C467FB0200E9
:1004700000000004595A504F52514A4D4B4E2A4CDD
:100480002F30B6B7ABACBBBCA9AABDBECFD0CDCECA
:10049000DBDCD9DA0D0E0B0F1A0508050905071864
:1004A00011130408120C11241FBECFEFDAE0DEBFD7
:1004B000CDBF04B603FE18C08091120590911305BC
:1004C000A0911405B09115058730904BA740B04B13
:1004D00059F41092120510921305109214051092FF
:1004E0001505E0E0F8E3099511E0A0E0B1E0E4E9EA
:1004F000F5E602C005900D92A03BB107D9F725E0C3
:10050000A0EBB1E001C01D92A231B207E1F70E9459
:10051000E2240C94553274CDA4E0B0E0E2E9F2E0BC
:100520000C94D02F2C01FB013A0129833A830B83D1
:100530001C831701960185017401898C9A8C808136
:1005400091814816590614F451824082D301CD900E
:10055000DC901197C414D5041CF44D925C92620196
:10056000A080B180C6018A199B098A309105ECF1FF
:1005700063E070E00E941B306A0D7B1D4616570633
:100580000CF07BC0AB81BC818C91811509F470C0EB
:10059000D7018D919C91DC01AA0FBB1FA20FB31F45
:1005A000CD92DC92D7018D919C9111978E3191055E
:1005B0000CF057C001968D939C9340815181D301DB
:1005C0008D919C91841B950B97FD01969595879530
:1005D000840F951F91838083D3018D939C93A98170
:1005E000BA811C92AB81BC811C92AB8DBC8D8C916D
:1005F000811509F466C0D901225C3F4F80E090E08C
:100600004D915D91840F951F2A173B07C9F76FE144
:1006100070E00E941B309B01D4018C91811509F47C
:1006200069C0F101A101425C5F4F80E090E06191FF
:100630007191860F971F4E175F07C9F76FE170E042
:100640000E941B30FB01C9018E1B9F0B63E070E011
:100650000E941B30CB018E0F9F1F2496E2E10C9469
:10066000EC2F1D921C9281E0AB8DBC8D8C93A5CF9D
:1006700081E0A981BA818C93B8CF641575050CF01F
:10068000B4CFA981BA818C918115B9F0D8018D912F
:100690009C91DC01AA0FBB1FA20DB31DAD92BC92B1
:1006A000D8018D919C9111978E3191050CF482CFD8
:1006B0001D921C9281E0D401D9CF81E0AB81BC8135
:1006C000DACFD7016D917C91D90120E030E080E054
:1006D00090E06115710551F4D3012D913C919CCFAF
:1006E0004D915D91840F951F2F5F3F4F2617370760
:1006F000BCF38FCFD8016D917C916115710581F0AC
:10070000F10140E050E080E090E0461757070CF020
:1007100097CFA191B1918A0F9B1F4F5F5F4FF5CF8C
:100720000190F081E02D8FCF9C01FB019A958115FE
:100730009F4120F5832F8170B32FB270AA27732FAA
:1007400074706627532F5870442734FF0DC082956C
:10075000807FAB2B09F08062672B09F08064452B0A
:1007600009F0806809950895AB2B09F08260672B2A
:1007700009F08460452BB1F38860F4CF80E0F2CFBC
:100780000C9434300895982F92959F7024E0911125
:1007900002C020E0982F892F86958695811511F04B
:1007A0002E5F982F892F8695820F089580930805D4
:1007B000089580930905089521E030E001C0220FDB
:1007C0008A95EAF780910905822BF3CF21E030E08A
:1007D000A90102C0440F551F8A95E2F7CA0180950E
:1007E000909109058923E5CF911121C08830F8F453
:1007F00091E001C0990F8A95EAF7892FE3EDF3E0C4
:1008000040E050E070E09191DF019B01042E02C0B6
:10081000369527950A94E2F72170219529272823F8
:1008200029272E934F5F5F4F4330510561F708959D
:10083000682F892F91111CC06830D8F4E3EDF3E0E4
:1008400040E050E0219130E0062E02C03695279519
:100850000A94E2F721703327042E01C0220F0A9474
:10086000EAF7822B4F5F5F4F4330510559F70895E8
:1008700080E008959091090521E030E0F90101C080
:10088000EE0F8A95EAF7D90102C0AA0FBB1F6A953D
:10089000E2F7EA2B01C0220F4A95EAF7892F8E234F
:1008A000E81303C0892F822B84CF2095822F8923C0
:1008B000FBCF8091810390918003981301C008952C
:1008C0008F5F8770FACF909154048095892380932D
:1008D0005404282F2770211110C0891771F09091AE
:1008E0000B0592FF0AC08695869586956FDF10925C
:1008F000540410925604109255040895982F909520
:10090000809151048923809351040895809150046B
:10091000811531F01092500410925804109257042F
:100920000895803E9105D9F1C8F48133910509F409
:1009300082C048F48932910509F472C08A32910567
:1009400009F480C0089589339105E9F08238910552
:10095000D1F08533910509F45EC00895843E910578
:10096000D9F148F4823E910539F1833E910549F170
:1009700081EE90E00895863E9105C9F1873E91058C
:1009800009F43EC0089520910A052370211164C026
:1009900020910B0523FF14C089E290E00895209177
:1009A0000A0520FD45C030910B0530FF09C024FD2C
:1009B00024C083EE90E0089520910A0522FDF7CF30
:1009C000089520910A0522FD44C030910B0530FDA9
:1009D00043C024FFF5CF11C020910B0521FFF0CFBC
:1009E00080910A0584FD09C087EE90E0089520916A
:1009F0000A0523FFE5CF24FFF7CF80E090E00895BC
:100A000020910A0523FD2BC030910B0531FFE1CF6A
:100A100084EE90E0089520910A0525FFD1CFBCCF48
:100A200020910A0525FD1EC020910B0523FFC8CF8C
:100A300089E390E0089520910A0526FFC1CF8AE25C
:100A400090E0089520910A0526FFBACF81E390E057
:100A5000089582EE90E0089580EE90E0089586EE8D
:100A600090E0089585E390E0089590910A0592FF43
:100A700010C041E0282F2471243009F040E031E01B
:100A8000282F2871283009F030E0431711F02CE0AE
:100A9000822793FF10C041E0282F2471243109F0F0
:100AA00040E031E0282F2871283109F030E0431769
:100AB00011F02CE0822730910B0530FF10C051E07F
:100AC000282F2171213009F050E041E0282F2871B2
:100AD000283009F040E0541711F029E0822731FF57
:100AE00010C041E0282F2171213109F040E031E0B0
:100AF000282F2871283109F030E0431711F029E040
:100B0000822794FD877E08951F93CF93DF9309DF9B
:100B1000EC01811522E5920708F052C0811540E5ED
:100B2000940708F0CDC0803E910520F58D3C9105DD
:100B300008F0A1C0883A910570F4853A910508F053
:100B400097C081309105B9F10497813A910598F1E8
:100B5000C0E0D0E030C0885A91094B97C8F7C85A16
:100B6000D0E0CC0FDD1FC55CDE4F0990D881C02DD1
:100B7000D46421C0811550E49507B0F4C11580E21A
:100B8000D80708F0B3C0C83ED105A8F0CE019A95A9
:100B900081159F41E8F68D2F68DF182FCE01992728
:100BA000C0DEEC01D12B07C09927BBDECC27DF705C
:100BB000C82BD92BD06ACE01DF91CF911F91089518
:100BC000803842E59407C8F5803652E5950708F06D
:100BD0005BC0C03482E5D807D0F4C03292E5D907B3
:100BE00008F04BC08C2F8695869520E2829FC0012D
:100BF0001124C37021E030E0A90102C0440F551F49
:100C0000CA95E2F7EA01C82BD92BDD68D4CF8C2F27
:100C100086958695877050E2859FC0011124C37028
:100C200021E030E0A90102C0440F551FCA95E2F748
:100C3000EA01C82BD92BDC68BECF803C52E5950772
:100C400058F48F71C03AD245A0F590E0982F8827CC
:100C5000EC01C46FD06AAFCF805C9245809708F0FA
:100C600077CFDC2FCC27CC27DF71C06FD06AA3CF22
:100C7000A497D064A0CFD0659ECFCF71D0E0DC2FF9
:100C8000CC27C16FD06A97CF86958695877020E272
:100C9000829FC0011124C37021E030E0A90102C08D
:100CA000440F551FCA95E2F7EA01C82BD92BDA6821
:100CB00082CFDBDEC82FD0E0DC2FCC27D0627BCF09
:100CC0008F71D3DE93E0CC0FDD1F9A95E1F7CC272F
:100CD000DF70282F30E084FF05C050E1859F900130
:100CE00011243327C22BD32BD06965CF8D2F8F7161
:100CF000BCDE182FCE01992714DEEC01D12BDECFFC
:100D000080E00895FB01811520E2920728F4811507
:100D100041E0940738F408959C0130522115304386
:100D200048F00895392F94FF02C03295307F20811A
:100D3000232B208399270895462B22FF0FC0982F3D
:100D400092959F708F70892B962F92959F706F70E0
:100D5000692B942F92959F704F70492B982F962353
:100D6000961309C050E04095509590E048235923D0
:100D700081E0452B09F080E0089510929A041092CA
:100D80009904E9E5F4E08581811102C0148216829C
:100D9000379684E0E139F807B1F70895AC01309156
:100DA0009C0460919B04232F621301C00895822F3D
:100DB00090E0FC01EE0FFF1FEF56FB4F0190F0811A
:100DC000E02DE417F50791F467E0649FF001659F5B
:100DD000F00D1124E75AFB4F41E044832313E6CF83
:100DE00001968370992780939C0408950196282F7B
:100DF0002370DACF0F931F93CF9301E010E0082EFA
:100E000001C0000F0A94EAF7C0914F049C2F902371
:100E1000911115C0909154049695969596958913C5
:100E200006C0109254041092560410925504C4DC6B
:100E3000C027C0934F04CF911F910F910895C6DC36
:100E4000F7CF282F35EB2303C001112497FF04C0EF
:100E500080589109892F089580589F4FFBCF80912A
:100E6000D80380FD14C081FD14C082FD16C080919E
:100E7000D703811581F08E3180F420E5829FC00177
:100E800011246EE170E00E941B30862F089584E1EA
:100E9000089588E2089588E0089580E50895809196
:100EA000D80380FD17C081FD17C082FD19C0809155
:100EB000D603811599F0883298F428E0829FC0010A
:100EC000112468E270E00E941B306115710551F039
:100ED000862F089562E0FCCF64E0FACF61E0F8CF9E
:100EE00068E0F6CF81E0089590913A04890290017C
:100EF000112437FF03C080933A0408952F3731053A
:100F00001CF4980F90933A0408959C0180E090E0BF
:100F1000F901E80FF91FE491E41307C091E0892774
:100F2000F901E80FF11D849108950196861780F369
:100F300080E00895E0917603F0917703309739F0DF
:100F40000190F081E02D309711F00995089580E02F
:100F50000895DC01E0917603F0917703309759F022
:100F600086819781892B39F082E08C930680F78106
:100F7000E02DCD0109950895A3E0B0E0E2ECF7E0A3
:100F80000C94E02F9C018091D8019091D901821797
:100F90009307B1F03093D9012093D801E091760303
:100FA000F0917703309761F00084F185E02D309760
:100FB00039F083E089833B832A83CE01019609952A
:100FC0002396E2E00C94FC2FA3E0B0E0EAEEF7E019
:100FD0000C94E02F9C018091D6019091D70182174B
:100FE0009307B1F03093D7012093D601E0917603B7
:100FF000F0917703309761F00084F185E02D309710
:1010000039F084E089833B832A83CE0101960995D8
:101010002396E2E00C94FC2F9C01FC0132968FEFAA
:1010200090E04191461751F08F3F19F4411101C0F2
:10103000892F9F5F9630A9F78F3F09F40895280FF5
:10104000311D87FD3A95F901628308959C01FC01E9
:101050003296285F3F4F8191861302C0DF011E92B6
:10106000E217F307C1F70895DC01FB0111969C918B
:1010700011978181981322C012968C911297811535
:1010800019F0928189131AC013968C9113978115C8
:1010900019F09381891312C015968C9115978115BB
:1010A00019F0958189130AC014969C91911521F02D
:1010B00081E02481291303C080E001C081E08170B8
:1010C00008958091010108952FB7F8946091D2019D
:1010D0007091D3018091D4019091D5012FBF0895D3
:1010E0000895FC019B018091C8019091C901861768
:1010F000970740F0672B29F48091E8008E77809362
:10110000E800C90140E0009741F4411106C0809118
:10111000E80082FF2FC080E0089520916F03211521
:10112000A9F12530A9F12091E80023FD2DC02091DF
:10113000E80022FDECCF2091E80020FFE4CF3091C1
:10114000F3002091F200009719F02830310558F093
:1011500041E02830310509F040E02091E8002E7789
:101160002093E800D0CF41914093F10001972F5F89
:101170003F4FE9CF80916F03811541F0853041F0F9
:101180008091E80083FFC3CF81E0089582E0089555
:1011900083E008958091C20187FF13C08091E80029
:1011A00082FF06C08091E8008B778093E800089565
:1011B00080916F038111F2CF089580916F038115A3
:1011C000D9F38091E80080FFF8CF8091E8008E7716
:1011D000ECCF2091E4003091E50095E6A901209143
:1011E000EC00822F817020FF06C08091E80080FF14
:1011F00006C080E008952091E80022FD1AC0809189
:101200006F03811589F0853089F08091EB0085FDB1
:101210000FC02091E4003091E50042175307F9F226
:101220009A95E1F684E0089582E0089583E00895B8
:1012300081E00895E8EDF0E080818E7F8083109258
:10124000E2001092DA001092E100A0EEB0E08C9182
:1012500081608C9380818F77808319BCA7EDB0E08B
:101260008C918E7F8C9380818F7E80831092C101C0
:101270000895E0917603F0917703309739F0028476
:10128000F385E02D309711F060E209950895982FCD
:101290009093E900891771F07091EC002091ED00B6
:1012A0005091F00021FD09C09F5F973089F780932E
:1012B000E9000895762F242F50E03091EB003E7F17
:1012C0003093EB003091ED003D7F3093ED00309195
:1012D000EB0031603093EB007093EC002093ED0055
:1012E0005093F0002091EE0027FDDECF0895A0E09E
:1012F000B0E0EDE7F9E00C94DA2FC8EDD0E088819A
:101300008F7E8883E7EDF0E080818160808384E0D8
:1013100082BF81E08093C10188818E7F888302EE45
:1013200010E0F80110821092DA0081EEC82ED12C64
:10133000F601108288818F7788838881806888830E
:1013400088818F7D888319BC10926F031092C00131
:1013500010923E021092BF0190EEE92EF12CF7019F
:1013600080818B7F808388818160888342E060E018
:1013700080E08DDFF60180818E7F8083F80180819F
:1013800081608083808188608083F70180818E7F87
:101390008083888180618883CDB7DEB7E8E00C94D4
:1013A000F62FE09181039091800329E0E91302C0B8
:1013B00080E00895AE2FB0E02E9FF0011124EE578B
:1013C000FC4F3181361306C03081381303C035819C
:1013D000341304C0FD013196E770E8CF81E0089531
:1013E00010920C0540910C0550910D0560910E0571
:1013F00070910F058FE090E00E94AB3040E050E02C
:10140000BA0183E190E00C94AB3081E08093E0007E
:1014100080E28093D8001092C9008FE097E2019794
:10142000F1F700C0000087E090EBDC01809312052B
:1014300090931305A0931405B093150588E19CE0E3
:101440000FB6F894A895809360000FBE909360004B
:10145000FFCF0F931F93CF93DF938B01EA019091FE
:101460006F03943051F58093E9008FEF9091E8007D
:1014700095FD06C09AE69A95F1F700C08A95B1F7F6
:101480008091E80085FF19C0A4DE811111C0809110
:10149000E80085FD06C08091E8008E778093E80023
:1014A000F3CFF80181918F018093F100219779F7B3
:1014B0008091E8008E778093E800DF91CF911F91B3
:1014C0000F910895792F603229F440E250E0682F9F
:1014D00082E0BFCF0895CF93DF93D82FC92F48E084
:1014E00050E0682F792F81E0B4DF88E0ED2FFC2FEA
:1014F000AAECB1E001900D928A95E1F7DF91CF91CE
:101500000895BC0146E050E084E0A3CFBC0143E075
:1015100050E084E09ECF90910B0592FB222720F9AA
:10152000281771F080FB92F990930B0560910A05E2
:1015300070910B0584E090E00E94B33082E0C3C953
:1015400008951F93CF93DF93962F122F632F84302C
:10155000A8F4911113C0483088F490E1899FE0010C
:101560001124C40FD11DC40FD11DCE0189960E9434
:101570009930612FCE018A960E949930DF91CF91E8
:101580001F910895CF9366E372E08FED93E06CDDD9
:10159000C82F811519F08FED93E0DBDC9091E0030B
:1015A00086E0EFEDF3E0DF01282F1D922A95E9F7A1
:1015B0009093E003A6E3B2E001900D928A95E1F7E3
:1015C00081E0911101C080E08C2BCF910895A4E2BD
:1015D000B0E0EDEEFAE00C94D42F4091DF0350918F
:1015E000E0036091E1037091E2038091E303909145
:1015F000E40307D42093DF033093E0034093E10337
:101600005093E2036093E3037093E40386E0EFED0D
:10161000F3E0DE01179601900D928A95E1F786E0DE
:10162000FE013796DE011D9601900D928A95E1F735
:1016300026E0FE013D96CE010196DC0101900D925F
:101640002A95E1F726E0FC01AFEDB3E001900D92A1
:101650002A95E1F726E0EFEDF3E0DE011796019021
:101660000D922A95E1F726E0FE013796DE015396AA
:1016700001900D922A95E1F726E0FE017396DC01B8
:1016800001900D922A95E1F726E0FC01AFEDB3E061
:1016900001900D922A95E1F726E0EFEDF3E0DE01EF
:1016A0005F9601900D922A95E1F76091E103F09029
:1016B000E20320914504D82EE92E0091E303109116
:1016C000E403211509F46DC0062E000C770B880B7E
:1016D000990B0E94663120E030E040E05EE30E941A
:1016E000F231209131023091320240913302509117
:1016F00034020E94CF303B014C016F2DFF0C770B61
:10170000880B990B0E94663120E030E040E05EE3F8
:101710000E94F23120912D0230912E0240912F0231
:10172000509130020E94CF305B01C82EF92EB301D8
:10173000C4010E943331162FB5018C2D9F2D0E94BC
:101740003331062F612F012E000C770B880B990B7C
:101750000E9466319B01AC01B301C4010E94CE30EE
:10176000609331027093320280933302909334027B
:10177000602F002E000C770B880B990B0E946631AE
:101780009B01AC01B5018C2D9F2D0E94CE30609342
:101790002D0270932E0280932F0290933002F12C31
:1017A00060E069A3FAA20BA31CA386E0FE017F966A
:1017B000DE01179601900D928A95E1F786E0FE0111
:1017C0003796AD2DBE2D01900D928A95E1F786E0FA
:1017D000ED2DFE2DDE01599601900D928A95E1F7CF
:1017E00086E0FE017996DE01179601900D928A95AA
:1017F000E1F786E0FE013796AFEDB3E001900D9280
:101800008A95E1F786E0E9EDF3E0DE0117960190B5
:101810000D928A95E1F78091E0039885892B80935A
:10182000E003B0DE811102C08091350210923502D2
:10183000A496EEE00C94F02F0F931F93CF93DF93B9
:10184000843000F561111EC04830E0F420E1829F31
:1018500080011124040F111D040F111DC801899668
:101860000E947830C82FD0E0DC2FCC27C8018A96A0
:101870000E9478309E01282BC901DF91CF911F91E2
:101880000F91089580E090E0F8CF462F20917203E9
:1018900030917303232B89F4703F39F4603F69F46E
:1018A00080917003909171030895711106C06830A2
:1018B00020F4843010F460E0BFCF80E090E0089521
:1018C000A0E0B0E0E6E6FCE00C94DB2F7C010091A8
:1018D000090580910805082BC3E0D0E010E0C8019D
:1018E0000C2E02C0959587950A94E2F780FD09C0F9
:1018F0002197A8F7D12C8D2DCDB7DEB7E7E00C945A
:10190000F72FDC2EB7018C2FC0DFFED8019781F3B3
:10191000F2CF0F931F93CF93FC018781908500979F
:1019200089F4858100811181811581F0611571F043
:10193000C801C6DFC82F682FC8010E94F403B80190
:101940008C2FA3DFCF911F910F910895C8010E94A2
:101950001804C82FF4CFCF93DF93D82FC92FB0DF4F
:101960006D2F7C2F92DFD0D8DF91CF910895FC01AD
:1019700084818115A9F087819085009799F0C4D85A
:10198000282F92959F709630B9F080F4925F9F70E7
:10199000923030F4203FD1F058F481E0283E58F0E6
:1019A00080E0089580819181D6DFEACF9A5FEFCF02
:1019B00081E0243FA9F7089591E0813F09F090E08C
:1019C00081E0283E08F080E0892B089581E00895A9
:1019D000382F292FCB01A32FB22F873023E0920776
:1019E000A105B10520F487509F4F0C94783080E01A
:1019F000089585E290E00E947830813C89F486E287
:101A000090E00E947830853C59F487E290E00E9493
:101A1000783091E0893509F090E0892F8170089540
:101A200080E0FCCFAAE0B0E0E8E1FDE00C94DA2F22
:101A3000EBEDF1E080E5DF011D928A95E9F7E9E53C
:101A4000F4E088E3DF011D928A95E9F78BEDC82E5B
:101A500081E0D82E7F0109E710E0F701D182C08232
:101A60004AE050E0B801CE0101960E94683088E05B
:101A7000FE013196D60101900D928A95E1F7898594
:101A80009A85D70113969C938E931297BAE0CB0E4A
:101A9000D11CE7E0EE0EF11C065F1F4F093C11055B
:101AA000E1F62A96E8E00C94F62FA6E0B0E0EBE52C
:101AB000FDE00C94DB2F0FEE13E089ECE82EF12C07
:101AC00098E0D92E46E050E0B701CE0101960E9481
:101AD0006830F8018D2D11928A95E9F7B8016C5F95
:101AE0007F4F89819A810ED9F80191838083B80153
:101AF0006B5F7F4F8B819C8105D9F8019383828333
:101B00008D8186838E818783F6E0EF0EF11C085F5E
:101B10001F4F89EFE816F104A9F62696E7E00C942A
:101B2000F72FAAE0B0E0E7E9FDE00C94DA2FC090CF
:101B30006D03D0906E0381E090E090936E038093EC
:101B40006D0310E08AEEE82E82E0F82E00E021E03E
:101B500030E0111104C0F701859195919C01402F4F
:101B600060E0812FEEDC0F5F82E0E80EF11C0830B0
:101B700071F71F5F143031F7FE0131967F018AE063
:101B800011928A95E9F709E710E04AE050E0B801C0
:101B9000C7010E94B730065F1F4F093C1105A9F726
:101BA00086E0F70111928A95E9F746E050E0B80126
:101BB000C7010E94B7300A5F1F4F093F1105A9F7FF
:101BC000D0926E03C0926D032A96E8E00C94F62F33
:101BD000A0E1B0E0EEEEFDE00C94D22FFE013196D4
:101BE00080E1DF011D928A95E9F701E310E099EFAA
:101BF000A92EB12C27E0422E23E0522E612C712C0D
:101C00004F0173016201B1E14B165104610471048B
:101C10001CF080E1C82ED12CA601B501C4010E94A0
:101C20008A30AC0CBD1C0D2C000CEE08FF084C18C3
:101C30005D086E087F080150104019F76096E0E1DA
:101C40000C94EE2F6FEF85E290E00E9499306FEFD9
:101C500086E290E00E9499306FEF87E290E00E9468
:101C6000993060E088E290E00E9499305ADFB0DF5E
:101C700061EC85E290E00E94993065EC86E290E0AC
:101C80000E94993069E587E290E00C949930CF93F7
:101C900024E030E043E060E080E30E94292FC82F79
:101CA000811105C00E949E2F8C2FCF91089582E054
:101CB0008A95F1F700C0F8CFCF93C82FE8DF8115E0
:101CC000C9F08C2F0E943B2F8FE391E00197F1F731
:101CD00000C000000E94532FC82F92E09A95F1F7A0
:101CE00000C00E949E2F82E38A95F1F700C08C2FDE
:101CF000CF910895C0E0FBCFA2E0B0E0E2E8FEE0C3
:101D00000C94DD2F182FF62EC2DF082F811106C08C
:101D100000E0802F2296E5E00C94F92F103511F0A9
:101D200010922B0210681983FA8262E070E0CE01F3
:101D300001960E946B2F892B59F78DE58A95F1F753
:101D400000000E949E2F81E291E00197F1F700C010
:101D50000000DFCF60E08436910550F067E78434FF
:101D60002FE2920728F464E670E00E940730615089
:101D70008FE0C2CF0E94942E8ADF811509F440C003
:101D80002AE62A95F1F700C00E949E2F8AE68A95DE
:101D9000F1F700C06AE58AE3AFDF811589F19FE7BB
:101DA00028E381E0915020408040E1F700C000002E
:101DB00082E082DF83E080DF84E07EDF85E07CDF1D
:101DC00086E07ADF0E949E2F8FE19EE40197F1F773
:101DD00000C000006FE08FE08FDF8FEC97E001978D
:101DE000F1F700C0000060E080E186DF60E081E1A3
:101DF00083DF62E083E680DF80E05EDF8FE35CCF3D
:101E00000895A8E1B0E0E7E0FFE00C94DE2F4B8BF3
:101E10005C8B6D8B7E8B8F8B988FFE01379686E067
:101E2000DF011D928A95E9F780912B028F018111C4
:101E300008C060E080E560DF811539F181E08093C2
:101E40002B0225DF811509F180E50E943B2FBDE5BE
:101E5000BA95F1F7000066E070E0C8010E94842F97
:101E60008F818770811110922B020E949E2F89858D
:101E70009A859195819591099A8789878B859C850B
:101E80009195819591099C878B8786E0FE01379615
:101E9000DE01119601900D928A95E1F786E0FE0130
:101EA0003196DE011D9601900D928A95E1F78D85A0
:101EB00083FD05C0898187FD17C010922C0286E042
:101EC000FE017396DE01179601900D928A95E1F757
:101ED0002F81388549855A856B857C8580E090E027
:101EE0006896E4E00C94FA2F4B815C812D813E8151
:101EF00080912C02811103C081E080932C02842FF9
:101F0000403851054CF08FE78D8B822F20383105FA
:101F100044F08FE78E8BD3CF40385F4FACF780E82B
:101F2000F3CF20383F4FB4F780E8F4CF1F921FB6AD
:101F30001F9211248F939F93AF93BF9380913D0283
:101F4000811113C08091D2019091D301A091D4014D
:101F5000B091D5014196A11DB11D8093D2019093FE
:101F6000D301A093D401B093D501BF91AF919F91BC
:101F70008F911F901FBE1F9018952FB7F8948091D6
:101F8000D2019091D301A091D401B091D5012FBF7E
:101F90000895CF93DF93C091510480915304C82BCF
:101FA000809150048115F1F0E8DF209157043091C1
:101FB0005804821B930B8838934110F00E948604CA
:101FC000D091500420E084EB91E0FC013081019637
:101FD00031112F5F31E08A3B9307B9F721110E943D
:101FE0008604CD2BC093B20148E050E068E773E06F
:101FF00082EB91E00E945430892BB9F088E0E2EB4B
:10200000F1E0A8E7B3E001900D928A95E1F7E09145
:102010007603F0917703309741F00280F381E02D51
:10202000309719F082EB91E00995DF91CF910895F7
:10203000811531F090915104892B80935104A9CFDF
:102040000895811519F00E947E04A3CF089581158B
:1020500031F090915304892B809353049ACF0895C3
:10206000811539F08095909153048923809353040E
:1020700090CF089580914904811521F082E2F0DF2C
:10208000109249040895962F20910B0522FF0FC04E
:10209000682F660F660F660F692B609354040E94C9
:1020A000DC036BDF909356048093550408950C94E1
:1020B000DC0390915004292F2823211559F0809595
:1020C000892380935004811531F057DF80935704A2
:1020D00090935804089580E090E0F8CF4EDF20916F
:1020E000DB033091DC03232B211521F08093650362
:1020F000909366032091DD033091DE03232B21159D
:1021000021F0809363039093640389ED93E00C9432
:10211000A907611509F45DC0E3E3E80FE33150F46A
:10212000F0E0E95AFD4C0C942E300E942F07819567
:102130008093DC03D3CF0E942F07FACF0E942F0792
:1021400081958093DB03F6CF0E942F07FACF0E9480
:102150004F078093DD03EECF0E944F078195F9CFA3
:102160000E944F0781958093DE03E4CF0E944F07C2
:10217000FACF282F215D330BA90121E030E001C007
:10218000220F4A95EAF79091DA03922B9093DA03A3
:102190004091E003815D21E030E0F90102C0EE0FE3
:1021A000FF1F8A95E2F7CF01611509F48CC0842BDB
:1021B0008093E003E7C98091D80381608093D803BE
:1021C000B9CF8091D8038260F9CF8091D803846021
:1021D000F5CF9091DB03482F50E08D3C59F42091CE
:1021E000DC0327FF0DC01092DC0391110BC010928D
:1021F000D70308C08E3CB1F42091DC0312169CF387
:102200009115B1F09091DD032091DE03922B911195
:1022100002C01092D603415D51094830510508F4BF
:10222000B7CF88CF8F3C39F497FFEACF1092DB030A
:102230009091DC03DACF803D19F41916BCF3E0CF9E
:102240002091DD03893D29F41216D4F61092DD03A6
:10225000D7CF8A3D19F427FFD3CFF8CF2091DE03E3
:102260008B3D29F427FFCCCF1092DE03C9CF8C3DE4
:1022700019F41216CCF3C4CF2FE2280F283080F4C3
:10228000FA01E15DF10921E030E001C0220FEA9599
:10229000EAF720953091DA0323232093DA03B0CFB5
:1022A0002091D8032E7F8D3D59F02091D8032D7FAA
:1022B0008E3D31F08F3D09F0A3CF2091D8032B7FC5
:1022C0002093D8039DCF8095842372CFCF93C82FBE
:1022D0008115A9F08CEF8C0F813A98F4E4EBF1E0D2
:1022E0008AEB91E02191C21709F43DC08E179F0738
:1022F000C9F76C2F82EB91E00E940C084ADECF9167
:10230000089580E28C0F883068F4C77021E030E0D7
:1023100001C0220FCA95EAF780915104822B809365
:102320005104ECCF8BE58C0F833038F42C2F2452E2
:10233000330BC9010E94BC07E2CFE8E5EC0FEB319B
:1023400050F4F0E0EE0FFF1FEF58FE4F80819181B7
:102350000E94E407D4CF83E38C0F833180F661E0E1
:102360008C2FD7DECCCF6C2F82EB91E00E94260819
:1023700010DEBFCF811571F19CEF980F913A30F4C8
:10238000682F82EB91E00E94260803CE90E2980F1E
:10239000983050F4877091E001C0990F8A95EAF760
:1023A000892F0E947E04F1CF9BE5980F933020F493
:1023B00080E090E00C94BC0798E5980F9B3120F4E6
:1023C00080E090E00C94E40793E3980F933110F4CD
:1023D00060E09FCE08951F93CF93DF93182FEB01FA
:1023E00075DF209731F4812FC5DFDF91CF911F91E9
:1023F00008958FEC97E00197F1F700C00000219756
:10240000F0CF60E570E0893311F060E070E0E3CF79
:10241000A0E0B0E0EEE0F2E10C94D92FEC0188816D
:102420008115D9F0813009F03FC08981813021F4D4
:102430008A812396E6DFF3CF823021F48A812396C6
:1024400045DFEDCF833021F48A81239693DFE7CFF8
:10245000843041F022968111E2CFCDB7DEB7E9E0BA
:102460000C94F52F8A81239620E030E09AE0682FC3
:102470006053770BAB016A30710560F021153105AF
:1024800051F3EFECF7E03197F1F700C00000215075
:102490003109F4CF929FB001939F700D11249A01DE
:1024A000260F371F8991E3CFE82FF0E0E354FE4F6A
:1024B000B490282F26952695269530E0F901E3550E
:1024C000FE4FE4908770F12C082E02C0F594E7943B
:1024D0000A94E2F7E0FAEE24FF24E0F8F901E3566B
:1024E000FE4FC490D12C082E02C0D594C7940A94F4
:1024F000E2F7C0FACC24DD24C0F8F901E357FE4F1F
:10250000049110E002C0159507958A95E2F70170D5
:102510001127E114F10411F081EED8DEC114D104C9
:1025200011F086EED3DE60E070E08B2D54DFC11435
:10253000D10411F086EE1EDFE114F10411F081EEFA
:1025400019DF0115110511F08CE25BDF219667CFD1
:10255000CF9310925104C6E0E4EBF1E0DF018C2F41
:102560001D928A95E9F780E090E00E94BC0780E028
:1025700090E00E94E407109253040BDDE9EDF3E0D4
:10258000DF011D92CA95E9F71092D7031092D60386
:102590001092D803A3DDCF910895DADF2FE78AE107
:1025A00096E0215080409040E1F700C0000088E1B3
:1025B0009CE00FB6F894A895809360000FBE9093AE
:1025C0006000FFCFAAE2B0E0E8EEF2E10C94DF2F6A
:1025D00082EC91E0FC0101962091F100208321E042
:1025E0008A3C9207B9F78091C301893009F459C038
:1025F000C8F4823009F4B6C0833009F485C0813054
:1026000089F18091E80083FFEAC08091C201909136
:10261000C3019A3008F0E3C0E92FF0E0E659FD4C21
:102620000C942E308A3009F48CC08B3051F7809195
:10263000C201813231F78091C6019091C701892B87
:1026400001F78091E800877F8093E8000E94CA0824
:1026500081E09091C401911101C080E0809302015A
:1026600077DFCFCF8091C201813A59F68091E8009F
:10267000877F8093E8008091C6019091C701892BE4
:1026800061F060E080E090E070E00E94710880916D
:10269000E8008B778093E800B4CF68E08AEC91E0A3
:1026A000F3CF8091C201813209F0ABCF8091C60196
:1026B0009091C7018D7F892B09F0A3CF8091E8000D
:1026C000877F8093E8008091E80082FF18C0909196
:1026D000F3008091F200029731F48091F100813093
:1026E00011F0863021F48091F100809301018091F6
:1026F000E8008B778093E8000E94CA0882CF80911F
:102700006F038111E0CF7DCF8091C201813A09F042
:1027100078CF8091C6019091C701892B09F071CFC4
:102720008091E800877F8093E8008091E80080FF37
:10273000FCCF809102018093F1008091E8008E77B8
:10274000D9CF8091C201813209F05BCF8091E8003E
:10275000877F8093E8000E94CA088091C50180931A
:1027600000014FCF8091C201813A09F04ACF809198
:10277000E800877F8093E8008091E80080FFFCCF2D
:1027800080910001D8CF803889F0823841F580915E
:10279000C6018F70873018F58093E9008091EB00B7
:1027A00085FB882780F91092E90006C080913E02DF
:1027B000880F9091BF01892B9091E800977F9093AB
:1027C000E8008093F1001092F1008091E8008E778C
:1027D00023C0811116C08091C401813011F1809114
:1027E000E80083FF0AC08091E800877F8093E800BB
:1027F0008091EB0080628093EB00AA96E3E00C945A
:10280000FB2F823061F78091C401811589F010920D
:10281000E9008091E800877F8093E8000E94CA0861
:10282000DECF81E0933009F080E080933E02EFCF6D
:102830008091C6018F702FEF280F263080F680938D
:10284000E9002091EB0020FFE2CF933031F480913A
:10285000EB0080628093EB00DACF9091EB00906107
:102860009093EB0021E030E0A90102C0440F551F16
:102870008A95E2F74093EA001092EA008091EB001B
:102880008860E8CF8111ABCF1091C4011F77809190
:10289000E3008078812B8093E3008091E800877FBC
:1028A0008093E8000E94CA088091E80080FFFCCF76
:1028B0008091E30080688093E30083E0111101C000
:1028C00082E080936F038BCF8058823008F087CFEF
:1028D0008091C4019091C5018C3D53E0950799F515
:1028E00083E08A838AE289834FB7F894DE011396E6
:1028F00020E03EE051E2E32FF0E050935700849156
:1029000020FF03C082958F703F5F8F708A30C8F0C0
:10291000895C90E08D939D932F5F243161F74FBFC9
:102920008091E800877F8093E8006AE270E0CE0142
:1029300001960E9471088091E8008B778093E800EF
:102940004ECF805DE6CF292F33272330310509F4A0
:102950004EC078F52130310509F488C08BE590E050
:10296000EDE3F2E02230310509F039CF2091E800A3
:10297000277F2093E8002091C8013091C901821778
:10298000930708F49C0140E02115310509F073C05C
:10299000411171C08091E80082FDCDCF80916F031D
:1029A000811549F2853039F28091E80083FFF2CF3A
:1029B000C2CF8091C6019091C7012132310509F43F
:1029C00046C02232310509F00ACF8330910508F064
:1029D00006CFFC01EE0FFF1FE95DFE4F0190F08175
:1029E000E02D8C5D9E4FDC018C9190E010C09C012D
:1029F0003327823021F12330310568F4232BB9F4D9
:102A0000E6EEF2E0E4918E2F90E0E6EEF2E0009741
:102A100009F4E5CEABCF2330310509F0E0CEEAEA88
:102A2000F2E0E4918E2F90E0EAEAF2E0F0CFE6EDFA
:102A3000F2E0E4918E2F90E0E6EDF2E0E8CFE8ECF2
:102A4000F2E0E4918E2F90E0E8ECF2E0E0CF83300A
:102A5000910508F0C4CEFC01EE0FFF1FE35DFE4FB1
:102A60000190F081E02D89E090E080CF82E190E05C
:102A7000E8E9F2E07BCF80916F03811509F45BCF29
:102A8000853009F458CF8091E80083FD54CF8091C0
:102A9000E80082FD7FCF8091E80080FF75CF9091A4
:102AA000F3008091F2002115310519F0883091056D
:102AB00050F041E0089709F040E08091E8008E77FF
:102AC0008093E80061CF44914093F100319621500A
:102AD00031090196E8CF803809F081CE8091E80075
:102AE000877F8093E8008091C0018093F1006DCED4
:102AF000811175CE1091C401123008F070CE809112
:102B0000E800877F8093E8001093C0010E94CA0804
:102B10001115F9F084E080936F0342E061EC81E0ED
:102B20000E94470942E261EC84E00E94470942E2C8
:102B300061EC82E00E94470942E260EC83E00E947F
:102B4000470980916F03843051F482E08093030140
:102B500046CE8091E30087FDDDCF81E0DCCF81E0D0
:102B6000F5CFEF92FF920F931F93CF93DF93C62F72
:102B7000D42F122F811599F060934D04FED99093B4
:102B8000BE018093BD01C77081E001C0880FCA9566
:102B9000EAF74EDACDB7DEB7E6E00C94F82F809175
:102BA0004D0468132DC0E090BD01F090BE01E5D941
:102BB0008E199F09883C910518F500E20D0FCD177D
:102BC00099F0C770FF24F3948F2D01C0880FCA9528
:102BD000EAF737DA083040F48D2F877001C0FF0C18
:102BE0008A95EAF78F2D24DA812F0BDC083090F6D6
:102BF000D77081E001C0880FDA95EAF722DACACFF0
:102C0000C77081E001C0880FCA95EAF7F7CFA9E045
:102C1000B0E0EDE0F6E10C94D02F8C01DC011496CD
:102C20008C91811509F4FBC061E0C8010E94890CF8
:102C30007C0180914404811136C0F80185818115A1
:102C400009F4A2C0E114F0E5FF0608F086C0E11423
:102C500020E2F20608F0E7C0E11437E0F30619F1CC
:102C6000F0F4C701805E91090897E8F030915104B3
:102C7000809153042091500499E0F801A0E3B4E05E
:102C800001900D929A95E1F7F0923804E0923704A2
:102C900010923A04832B822B80932F0404C0E114FA
:102CA0005FE0F50619F7F8018081813071F4D801F1
:102CB00011968C91811109C060D99093480480933A
:102CC0004704F801858180934604D80115968C91BC
:102CD000E114BEE7FB0609F0A8C18115E1F080917F
:102CE0000C058F5F837080930C0540910C0550910B
:102CF0000D0560910E0570910F058FE090E00E9428
:102D0000AB30E0910C05F0E0EE0FFF1FE955FE4FF0
:102D1000808191811FD8D80115964C91411195C1A0
:102D200053E7E5165CE7F50609F468C0A2EAEA167F
:102D3000A2E5FA0609F4ACC208F081C2C7019052BC
:102D40008115904208F496C2B1EEEB16F10409F435
:102D50009FC2E5EEEE16F10476C290EEE91692E51A
:102D6000F90658F4A0E6EA16A2E5FA0608F09BCFA9
:102D7000C70192558034910578CF970127573C477A
:102D80002530310508F072CFF9E7EF16FCE7FF06B2
:102D900009F04DC02091370430913804232B71F194
:102DA000811599F081E00E94740780912F044FD91A
:102DB00089E0E0E3F4E0A6EEB3E001900D928A959D
:102DC000E1F780913A048093E50386E0F801A6EEEE
:102DD000B3E001900D928A95E1F78091E50380932D
:102DE000440486EE93E013DF10924404D801159654
:102DF0008C91811103C080912F0432D980915404A9
:102E00008770811561F0D80115968C91811539F084
:102E100080910B0582FF03C082E00E946304299623
:102E2000E2E10C94EC2FF801868180311ECFBAE7E5
:102E3000EB16BCE7FB0609F036CF811509F4CAC0D2
:102E4000A0903704B0903804E0912F04E887E9831C
:102E5000BE016F5F7F4FC5010E9482062C01F98180
:102E6000F9878FEEC82E83E0D82EEE24E394F12C60
:102E700022242A94D60117963C90179733FE54C00B
:102E80006D907C90119712968D909C90139746149C
:102E90005704B9F41496BC91BF83232DF6014681E3
:102EA0006B2F89850E949C06811559F08F810E94A5
:102EB000C003281634F4D60115969C917401F92AA2
:102EC000282E48145904C9F431FE17C0F601F581C3
:102ED000FF83232DD60116964C916F2F89850E9472
:102EE0009C06811551F08F810E94C00328162CF496
:102EF000F60194817301F92A282E30FE15C0FFEFE8
:102F00002F1212C021E0E216F10471F4232DD60134
:102F100016964C9160E089850E949C06811521F0EF
:102F2000F60185817401F82AF8E0CF0ED11C2FE25A
:102F300034E02C153D0509F09DCF31E0E316F10496
:102F4000F1F5988592959F704885942B9F7081E04C
:102F5000403108F480E0F82EF294B0EFFB22F92A19
:102F6000A11450E2B50620F5A11481E0B80608F0DE
:102F700055C0EA2C8F2D8D704A2D811509F451C052
:102F80006AE08CE994E00E948507282F30E0211543
:102F9000310551F44E2D6EE186E794E00E948507DD
:102FA000282F30E0811549F0F901FF297F0107C082
:102FB000C50190528115904390F1E12CF12C87E0EE
:102FC000EBE3F4E0DF011D928A95E9F7F092430408
:102FD000E09242048091420490914304892B09F4C9
:102FE0000DCFF8018581811539F08FEF0E947407AC
:102FF00080913A048093390486E0F801ABE3B4E0B1
:1030000001900D928A95E1F78091390480934404F0
:103010008BE394E0FCDD10924404F0CEFB28BB244B
:10302000A8CF68E084E994E0AECFE1E0EE16EEE7E9
:10303000FE0609F070CE811509F46DCE809145042D
:1030400091E089278093450466CEC7019757803861
:10305000910508F09DC6BE2CB0E1EB1608F0CECE6F
:1030600066E073E080E090E00E94E80C8111C6CE3B
:10307000C12CD12C7601B11047C074E0272E9E01DF
:103080002F5F3F4F3E832D83AD81BE81E22D1D9288
:10309000EA95E9F746015701FFEF8F1A9F0AAF0A39
:1030A000BF0AC701B6010E94E80C8983811509F4A3
:1030B000A5CE813009F0AFC02601370122E0420ED3
:1030C000511C611C711CC501B4010E94E80C382E12
:1030D0008A83811509F492CE8FEF830D833048F5F2
:1030E000C301B2010E94E80C8B83811519F0CE0157
:1030F00001968ED94601570133E0830E911CA11C25
:10310000B11C75016401C0CFE7E0CE16E3E0DE0636
:10311000E104F10409F472CEC701B6010E94E80C83
:10312000FFEFCF1ADF0AEF0AFF0A8111EDCFBA9441
:10313000A2CF8BEF830D8330B8F54601570143E0F2
:10314000840E911CA11CB11CC301B2010E94E80CA9
:103150008B838115B1F2C501B4010E94E80C8C8308
:10316000811108C04601570154E0850E911CA11C35
:10317000B11CC7CFAB80BC8081E0A8168FEFB8062A
:1031800010F0BA2CAA2496E0391651F0A7E03A16AE
:1031900019F0C5010E943224C5010E946424E2CFC7
:1031A000C5010E943224DECFB4E0530142013B123C
:1031B000A8CFC301B2010E94E80C782E4601570146
:1031C000E4E08E0E911CA11CB11CC701B6016D5F1D
:1031D0007F4F8F4F9F4F0E94E80C711409F40ECE61
:1031E000811509F40BCE8150990B4FEF489F900148
:1031F000499F300D1124472D4150550B240F351F89
:103200002150310908F47DCF8FEC97E00197F1F759
:1032100000C00000F5CFCE010196FAD872CF10920F
:1032200051040E9486040E94BD0F88579C4E9093C3
:103230004B0480934A0481E080934904DFCDF2EB94
:10324000EF16F2E5FF06E9F525EE30E027703327AB
:1032500081E090E001C0880F2A95EAF720914C04A4
:10326000309149043115E1F04115A9F0282B209344
:103270004C04C4CDD80116968C91803110F58F2D59
:1032800099278F7199278230910511F04297DBCFF2
:1032900021EE30E0DBCF8095822380934C04AECDCD
:1032A000322F3823311569F0982F909592239093FF
:1032B0004C040E947E04D80115968C91811509F466
:1032C0009DCD80914904811509F4D1C0C09051046D
:1032D000D09050040E94BD0F88579C4E90934B0491
:1032E00080934A04F8018581811509F4C0C08D2DB1
:1032F0008C298D79811190C0E114F0E5FF0608F565
:10330000E11420E4F20608F09BC036EEE316F10467
:1033100009F449C0C70190528115904208F097C046
:10332000D80116968C91803108F46EC0C701992798
:10333000109253048D32910509F582E08093530475
:103340008AC0B0EEEB16B2E5FB0608F04DC0E0EC2B
:10335000EE16E2E5FE0638F5F0EAEF16F2E5FF06B6
:10336000E8F420E6E21622E5F206E8F4C7019255F9
:1033700080349105C0F010925304C7018E3291053C
:1033800008F082C08832910508F063C08E31910543
:1033900008F061C004974A9780F23EC034EBE31610
:1033A00032E5F30641F7D80115969C91911509F481
:1033B000C4C410924D04970130572332310508F0F0
:1033C000CDC484E090E00E94853090930B058093FB
:1033D0000A05F701E150F047E232F10508F076C046
:1033E000EC58FD4C0C942E3049E7E4164CE7F406FB
:1033F00030F457E7E5165CE7F506A8F6BCCF8BE797
:10340000E8168CE7F806CECF8F2D8F71843159F2F4
:10341000863161F4109253040E943A108091510455
:1034200090914C04892B8093510421C00E943A1042
:103430008091510490914C04892B80935104B3CF17
:10344000D80116968C91803108F070CFACCFC701AF
:103450006FCF8A9709F780914C04811531F08091E4
:10346000530492E08927809353040E94C90FF80106
:103470008581F701E851FC47E730F10508F093CF6B
:10348000EA56FD4C0C942E308C34910521F38D328C
:103490009240E0CF26E241EE61EE63DBAFCC27E263
:1034A00045EE65EEFACF26E241EE60EEF6CF27E27A
:1034B00045EE64EEF2CF26E241EE62EEEECF27E279
:1034C00045EE66EEEACF28E241E0EBCF80910A05B7
:1034D000816080930A0560910A0570910B0584E074
:1034E00090E00E94B33034D889CC80910B0588607D
:1034F00080930B05F0CF80910A058260EACF80911E
:103500000A058460E6CF80910A058860E2CF809149
:103510000B058160EDCF80910B058260E9CF809132
:103520000A058061D6CF80910A058062D2CF809152
:103530000A058064CECF0CD880910A058068C9CF77
:1035400080910A058C60C5CF80910B058360D0CF38
:1035500080910A058E7FBDCF80910B05877FC8CFF4
:1035600080910A058D7FB5CF80910A058B7FB1CF01
:1035700080910A05877FADCF80910B058E7FB8CFF4
:1035800080910B058D7FB4CF80910A058F7EA1CFEE
:1035900080910A058F7D9DCF80910A058F7B99CF01
:1035A0000E94A81280910A058F7793CF80910A0517
:1035B000837F8FCF80910B058C7F9ACF80910A05F6
:1035C000992782FF939590FB82F990FB83F981CF35
:1035D00080910B05982F909590FB80F990FB81F9D5
:1035E00087CF90910A05892F8F7B96FF806471CFDA
:1035F0000E94A81290910A05892F97FB87F980589D
:1036000068CF61E08EE090E00E94993064CF60E086
:10361000F9CF90910A05892F8F7E94FF806159CF51
:1036200090910A05892F8E7F90FF816052CF9091F3
:103630000B05892F877F93FF88605ACFB7E7EB167A
:10364000BCE7FB0609F1E8E7EE16ECE7FE0639F108
:103650009701205E32452032310530F5911124C0AA
:10366000FE2DFF7181E090E09C0102C0220F331F0C
:10367000FA95E2F77901622F83E090E00E94993099
:103680008E2D0E94D603BACB81E0911551F00E9495
:10369000DC0343E062E081E00E943A04AFCB82E0C9
:1036A000F4CF0E94E603F5CF40914F0480910905C5
:1036B000282F30E02095309570E024233723232BEA
:1036C00019F0482340934F043BE7E3163CE7F30629
:1036D00041F4911509F492CB0E94C3030E94FA06AB
:1036E0008DCB40E4E41642E5F40608F05AC050E2FF
:1036F000E51652E5F50608F05BC0E11480E5F80632
:1037000070F5E114A0E4FA0608F068C0911509F418
:103710007DC0FAE5EF16FCE7FF0609F4D5C008F016
:10372000B7C031E0E3163CE7F30609F4CBC043E051
:10373000E4164CE7F40609F4BFC0E1145CE7F506B3
:1037400009F064C00E94A812AFE7BAE1E6E0A15018
:10375000B040E040E1F700C000000E94050A970178
:1037600030552115324090F6970145E03695279562
:103770004A95E1F7822F8F7020914F0430E041E0AD
:1037800050E0082E02C0440F551F0A94E2F724238C
:103790003523232B09F4BACF9111A0CF10925104F5
:1037A000F4C29701205C32452032310508F0AECFDB
:1037B0008E2D8F7120914F0430E041E050E0082EB3
:1037C00002C0440F551F0A94E2F724233523232B0C
:1037D00009F49CCF911509F411CB80CFF8018681B3
:1037E000803108F093CF911111C02F2D2F7081E0FF
:1037F00090E002C0880F991F2A95E2F720914F04AC
:1038000030E082239323892B09F0F8CAF8018781DD
:103810009085009709F45CC00E9484057C01F80142
:10382000B580A680A2942FE0A222809154048770D4
:10383000811509F1CB2CB114F9F08F2D807F8034E4
:1038400069F080E28E0D8830B0F08F2D807E80325E
:1038500029F4F2E0EF1678F0A11469F080910B05DD
:1038600082FF09C082E00E94630480915404877043
:10387000CC24C3948111C12CEF2DE295EF7020EC84
:10388000F21608F09EC0F0E0E356FD4C0C942E308A
:103890008BE5E8168CE7F806C9F080910B0500244B
:1038A00082FF0394802D9CE5E9169CE7F90609F058
:1038B000ADCF0E948B0AAACF6FEF7FEF80E090E040
:1038C0000E94B3300E94CD1281E0F3CF80E0F1CFAF
:1038D0008581C080D180811569F0C6010E94600C8D
:1038E000F82E682FC6010E94F403B6018F2D0E94A6
:1038F000450C92CFC6010E941804F82EF6CF3F2D3A
:103900003F70D32E40E1F41618F0D29490EFD922F4
:10391000B114B9F0D11469F080E28E0D883010F046
:10392000E11009C0809151048D29809351040E94B7
:10393000C90F8E2D44C0809153048D298093530468
:10394000F6CF8E2D0E94BA11D114D9F180E28E0DDE
:10395000883010F0E11004C08D2D0E947E0406C056
:10396000D094809153048D21809353040E94C90FF9
:1039700028C05F2D5F70D52E8F2D807F803219F08B
:10398000D29480EFD822E11451F081E0E81609F4D6
:1039900084C0B11409F490C0A114B1F1CACF8091D0
:1039A0000B0582FD2DC0B11429F1D11439F080919D
:1039B00051048D29809351040E94C90F80E00E9418
:1039C0006611C11409F4DAC08091540480FDD6C098
:1039D000D80115961C928695869586950E94DC03E3
:1039E000C80115D9809154048695869586950E94C4
:1039F000E603C4C080E00E94BA11D11411F3ACCF29
:103A0000B11469F1A11004C08D2D0E941810D9CFF6
:103A100091E0A91210C0F09050048D2D8F21D8167E
:103A200081F20E94BD0F9093580480935704FD28A3
:103A3000F0925004C6CFA5E0AA12C3CF8D2D0E94EC
:103A400018108D2D0E945910809152049D2D98239D
:103A5000D91609F4B6CF8D2980935204B2CFA110A4
:103A600012C08D2D0E9421108D2D0E945910809121
:103A700052049D2D9823911509F4A3CFD094D822F8
:103A8000D09252049ECFB1E0AB129BCF80915104F3
:103A90008D21811509F495CFE4CFB11429F0E6E02A
:103AA000AE1608F08ECFB0CFF5E0AF1608F089CF94
:103AB0008D2D0E94211085CFA114D1F329E3E212AC
:103AC00009C03FEF43EF51E0315040405040E1F733
:103AD00000C000008E2D0E94BA1173CF8F2D8695E5
:103AE00086958370811561F0813009F06ACFC70136
:103AF0009370B11002C080E090E00E94E40761CFB3
:103B0000C7019370B11002C080E090E00E94BC0732
:103B100058CF6B2D8E2D0E94891053CF8F2D83701F
:103B2000811139C0B11028C04E2D4295469547707D
:103B3000440F440F8E2D8F70042E01C0880F0A94FD
:103B4000EAF72E2D2071E4FE07C02FE030E001C01F
:103B5000220F4A95EAF720953F2D3695369533701A
:103B60003230A1F0333081F040910805313059F006
:103B7000822B84230E94D6030E949A0760E0C8012A
:103B80000E94890C4CC9842B822BF4CF822B9091FC
:103B900008058927EFCFB11459F1F0FEEDCF4E2D76
:103BA000429546954770440F440F8E2D8F70042E1A
:103BB00001C0880F0A94EAF72E2D2071E4FE07C099
:103BC0002FE030E001C0220F4A95EAF720953F2D03
:103BD000369536953370323089F0333069F0409144
:103BE0000905313041F0822B84230E94D903C4CFD0
:103BF000823010F2D4CF842B822BF7CF822B90917E
:103C000009058927F2CF8F2D8F70F82EB11431F06E
:103C10000E94DC038E2D0E941810AECF8E2D0E94C4
:103C200021108F2D0E94E603A7CF92EFE916A1F194
:103C3000A3EFEA1680F4B0EFEB16E1F0E1EFEE1639
:103C4000A1F0B11409F467C0A11409F461C08E2D6C
:103C50000E94661191CFF3EFEF1629F124EFE212E3
:103C6000F0CF80910B0582FD2AC08F2D8F71B1148A
:103C7000C9F216C0B11469F035E0A31608F07CCF84
:103C80002F2D2F7181E090E001C0880F2A95EAF76F
:103C9000B6CF46E0A416F2CF8F2D8F71B110C2CFF0
:103CA0000E94DC0369CF80E0B11409F49ECF9F2D00
:103CB0009F7181E001C0880F9A95EAF796CFB11401
:103CC000C1F0809154048770843049F410925404F8
:103CD00010925604109255048F2D8F71A3CF55E08A
:103CE00063E0A51608F048CF8F2D8F710E94431016
:103CF00043CF85E0A81640F0109254041092560469
:103D00001092550464E0F0CF81E00E94630434CF48
:103D10008F2D8F71C5CFA114F9F299E3E91209C073
:103D2000AFEFB3EFE1E0A150B040E040E1F700C0F9
:103D300000008E2D0E94BA111FCFF6E1EF16FCE7AE
:103D4000FF0609F07BCC80914E0465E3811101C030
:103D500069E282EB91E00E94260817C026E1E21694
:103D60002CE7F20609F06ACC809151048A7A91E03E
:103D7000811101C090E090934E0465E3811101C070
:103D800069E282EB91E00E940C080E94C90F36C8DC
:103D900033E7E3163CE7F30611F00C949616809196
:103DA0004904811509F43BCA0E943A1027C8809142
:103DB000D003803178F48091CF03811559F0E091E0
:103DC0008103209180033091CB034091CA0359E0D5
:103DD0002E1301C008956E2F70E05E9FF001112434
:103DE000DF01AE57BC4F14968C911497811559F191
:103DF00011968C911197831326C08C91841323C044
:103E000015968C91159781111EC012968D919C91DB
:103E1000A091CC03B091CD038A1B9B0B883C9105EC
:103E200090F48091D0038F7080618093D003E85725
:103E3000FC4F80818F70806180838AEC93E00E94C8
:103E400007160C945904FB013196E770C1CFAFE01F
:103E5000B0E0EDE2FFE10C94D42F8C0186E0F80194
:103E6000DE011A9601900D928A95E1F7F801F5802E
:103E700084819AEC892E93E0992E6090CE03611094
:103E800017C0811591F0F11409F43FC1C8010E94D7
:103E9000B70C811509F439C189E0F801AAECB3E047
:103EA00001900D928A95E1F782DFFF24F3945FC0C1
:103EB0007080A280B380D090CF032091CC0330914A
:103EC000CD03A501421B530BD11409F4E5C0483CB6
:103ED000510508F08CC0811541F38091CB03C1805E
:103EE000E090D00350E1E51608F062C0C8121EC091
:103EF0008091CA0387111AC02091D1033091D20357
:103F0000878190852817390789F4F1104BC08E2DD1
:103F10008F7080618093D0038AEC93E00E94071633
:103F20008091D003F8018683F12C21C0F1103AC0B2
:103F300040E06C2D872D0E94D10940E06C2D872D2B
:103F40000E94D109F82E8111EFCF8A859B850E94AE
:103F5000AB0C292F22952F70903470F49F70223073
:103F6000A0F09115B1F0F8019681903190F48F2D69
:103F70002F96EEE00C94F02F2A5F2F70223068F01D
:103F8000C8010E940716FD2CF2CF911511F0811582
:103F900071F3805E883058F3F3CF803F40F3815F48
:103FA0008330F9CF8091D00381608093D003BCCF60
:103FB000C8124EC08091CA0387114AC02091D10314
:103FC0003091D203878190852817390709F040C0C6
:103FD000F1103EC0E682C8010E94071689E0F80190
:103FE000AAECB3E001900D928A95E1F75ECFE090E4
:103FF000D003F0E1EF1650F48AEC93E00E9407162C
:1040000089E0F40111928A95E9F78ECF811509F4C0
:104010004CCF9091CB03F8018181981319C0809106
:10402000CA03871115C02091D1033091D203878133
:1040300090852817390761F4F1100AC0E682C8019B
:104040000E94071689E0F40111928A95E9F72DCFB5
:10405000C8010E94B70C811509F457C0F11409F486
:1040600054C08091D003803208F416CF8091CA03E7
:104070009091CB039A838983BC82AB826D821E822E
:10408000EF828091D1039091D20399878887CE01E6
:1040900001960E94071600CF483C510508F0B0CFAA
:1040A000811509F402CFF11481F19091CB03818144
:1040B000981321C08091CA0387111DC02091D1039C
:1040C0003091D2038781908528173907A1F4809118
:1040D000D00380FD83CF803108F480CF8683982F72
:1040E000907F903F09F477CF982F907F905F8F70EB
:1040F000892B868370CFC8010E94B70C8111CCCE6A
:104100008091D00381608093D003C8010E9407167C
:10411000CCCEA2E1B0E0EFE8F0E20C94DE2F0A870B
:104120001B872C873D874E875F87688B798B8A8BAF
:10413000CE010A968CDE811128C020918003309137
:10414000810389E0FE013A96DE01119601900D92FD
:104150008A95E1F78E858115C1F0822F90E0019656
:104160008770992738171906D9F099E0929FD001E6
:104170001124AE57BC4FFE01319601900D929A95D5
:10418000E1F7809380030E94590419E08091810334
:1041900090918003891312C06296E4E00C94FA2F88
:1041A0000E94A812109280031092810389E0EAEC29
:1041B000F3E0DF011D928A95E9F7E7CF189FC00170
:1041C00011248E579C4F43DE811531F3809181037A
:1041D00090E001968770992780938103D7CFEF9263
:1041E000FF920F931F93CF93DF9380910505E0918A
:1041F000DA01CDE0811130C0CDB7DEB7E6E00C9436
:10420000F82FD1E0DE0FD093DA01EE2EF12CCE9F05
:10421000F0011124E356FB4F84818115E1F0878181
:104220009085892B21F481859285019651F4008136
:104230001181228133814481558166817781808516
:1042400068DFCE9DF001CF9DF00D1124E356FB4FAA
:10425000148210925304ED2F80910505E81788F21F
:10426000109205051092DA01C7CFA4E0B0E0EBE3AD
:10427000F1E20C94D12F20919C04298397E0992E90
:1042800001E010E02DE0322E34E0532E8824839498
:1042900080919B049981891307C0A1DF0E94BD060C
:1042A0002496E1E10C94ED2F9981892F90E09C8375
:1042B0008B83FC01EE0FFF1FEF56FB4F8081918136
:1042C000989ED001999EB00D1124FD01E75AFB4F35
:1042D000FA83E983248121115BC060900505EDE933
:1042E000F4E060E070E0712C661508F04FC0A38424
:1042F000B484A981BA81CD90DC902FEF3FEF412C9F
:10430000442D50E07601E40CF11CE40CF11CD701C3
:10431000ED90FC90E114F10439F0AE14BF0409F003
:10432000A90143949A01ECCF2F3F3207D1F1D80174
:1043300002C0AA0FBB1F2A95E2F77A2A9801042C23
:1043400002C0220F331F0A94E2F7A901415051091C
:104350007416150629F5369EF001379EF00D1124CE
:10436000E356FB4F989ED001999EB00D1124A75A99
:10437000BB4F12962D913C9113973087278354821F
:10438000108211829287818715968C920E94CE06A8
:104390008B819C8101969A8389838370898378CFEE
:1043A00014826F5F7F4F3D969FCF1092070510924A
:1043B00006051092100180919B0480939C040E943A
:1043C000BD060DCFACE1B0E0E8EEF1E20C94D02FE9
:1043D0004B8B5C8B6D8B7E8B8F8BB92E988FA92E20
:1043E000911110925304188A198A1A8A86E0FE01E4
:1043F0007396DE011A9601900D928A95E1F75F8817
:1044000080910B0582FF1FC00E94BD0F20915504B3
:1044100030915604821B930B8838934138F0809179
:10442000540482FD03C082E00E9463040E94BD0F19
:104430002091570430915804821B930B8838934184
:1044400010F00E9486045114D9F05E86BF8661E0A8
:10445000CE010A960E94890C61E0CE010A960E9464
:10446000890C61E0CE010A960E94890C4C018035CE
:104470006CE7960791F4A11419F181E08093100183
:104480005E86BF860A851B852C853D85452D5B2D67
:10449000688979898A893DDECDC081359C4721F4C0
:1044A000A11471F082DFECCF82E588168CE79806C4
:1044B00039F4A11429F0809110018111F3CFDDCFDF
:1044C00049E5E42E44E0F42E412C612C712CD701F7
:1044D0006D917C91CC24CA94DD24DA9480E0282F5D
:1044E00030E0FB01E80FF11DE80FF11D4081518123
:1044F0004115510539F08416950609F096018F5F34
:104500006901EDCF10E0BFEFCB16DB0609F44EC01A
:10451000F701448110911001411110E0D701159667
:104520003C90159716969C911697A11409F405C115
:10453000111509F402C1311017C021E030E00C2C34
:1045400001C0220F0A94EAF7922B16969C932091B1
:10455000990430919A042233310530F422E330E09B
:1045600030939A0420939904E1E0F0E002C0EE0F4A
:10457000FF1F8A95E2F7CF010197D70116962C917C
:104580002817190699F4C0900605D0900705C114A4
:10459000D10409F453C00E94BD0F8C199D09C39723
:1045A00008F44CC081E0F701848311E0412ABFEF99
:1045B0006B1A7B0AE7E0EE0EF11CF8E06F1671044F
:1045C00009F085CFA11409F417C1411409F414C1ED
:1045D0000E94BD0F90930705809306058091050505
:1045E000883040F591E0980F9093050599E0FE0121
:1045F0003A96DE01119601900D929A95E1F75D824F
:10460000BE822DE0829FC001112483569B4F29E07A
:10461000FE013196DC0101900D922A95E1F72FEF12
:104620003FEFDC011A963C932E9319971C969C92AF
:104630008E921B976C96E2E10C94EC2F20919C04D7
:1046400080919B04922FE0E0F0E001E0281709F44C
:1046500048C0422F50E0FA01EE0FFF1FEF56FB4F0C
:104660002080318037E0329DF001339DF00D112420
:10467000E75AFB4F608171817C8F6B8FB0E030E037
:10468000A0E0EB8DFC8DEA0FF11DEA0FF11DC0805B
:10469000D180C114D104E1F0F7010190F081E02D47
:1046A000FA8FE98F30E007C0E1E0C616D70609F0BF
:1046B000E0E0BE2B3F5FE98DFA8DE30FF11DE30FC4
:1046C000F11D608171816115710571F7AF5FD9CFFF
:1046D000B11581F13A17C8F4E1E0D7011496EC93D3
:1046E000F70190939C04EE15FF0509F45FCF90E06D
:1046F000FC01EE0FFF1FEF56FB4F718260820196A7
:104700008370992780939B0451CF37E0329DF0014D
:10471000339DF00D1124E75AFB4F0483EE15FF057E
:10472000F9F2291302C09F5F93709A012F5F3F4FE8
:1047300023708CCFE0E0F0E0F8CF292F30E031108B
:1047400024C061E070E002C0660F771F8A95E2F72F
:10475000CB0101972817390791F010E0E1E0F0E074
:1047600002C0EE0FFF1FCA94E2F76F01C094D70199
:1047700016968C9116978C2116968C9317CF41150F
:1047800069F3C3010E94CE06E8CFA9010C2C02C038
:10479000559547950A94E2F7C9010197822393231F
:1047A000892B39F540FF25C0D70112968D919C9138
:1047B000892BD1F087E0FE013196DF011D928A95A9
:1047C000E9F70E94BD0F9C018B839C8384E08D835D
:1047D000F70192818381792F9887898709811A81CE
:1047E00044E05E816F8195DCD70115961C92132DF4
:1047F000B5CF142F1170B2CF90919C0480919B047F
:10480000981731F032DDB1E04B1609F413CF38CEF2
:10481000E6DC10920705109206050E94BD06F3CF54
:10482000A6E0B0E0E6E1F4E20C94DE2F0E94BD0FBA
:104830008C0180917403909175038017910771F03A
:1048400019821A820E94BD0FBC0149815A8180E001
:1048500090E0B8DD10937503009374032696E4E0AE
:104860000C94FA2FA6E0B0E0E8E3F4E20C94DE2F1B
:104870008C019093710380937003011580E21807F7
:10488000B0F4C801805E9109089728F067E270E1F2
:104890000115110511F468E170E1C8010E9494034B
:1048A000802F0E9466112696E4E00C94FA2F80EF88
:1048B00089838A830E94BD0F8160BC0149815A812E
:1048C00081E091E07FDDEFCFA6E0B0E0EAE6F4E240
:1048D0000C94DE2F8C01909371038093700301156B
:1048E00080E21807B0F4802F0E94BA11C801805EE0
:1048F0009109089728F060E370E10115110511F4A2
:1049000061E270E1C8010E9494032696E4E00C94F1
:10491000FA2F80EF89838A830E94BD0F8160BC01DA
:1049200049815A8181E090E04DDDEFCFCF93DF9355
:10493000A3E3B1E06BE371E041E030E02D912F3F64
:1049400079F0E22FE295EF70E05EF0E0808190E098
:104950002F7002C0959587952A95E2F780FF22C0B7
:1049600080E0382B440F6A177B0741F780913C02A7
:1049700083131AC08091BC01811509F1C091BA015D
:10498000D091BB010E94BD0F8C1B9D0B0597B8F009
:1049900080913C0290916C03891380936C03109278
:1049A000BC010DC0842FDDCF30933C0281E08093A9
:1049B000BC010E94BD0F9093BB018093BA01DF91AF
:1049C000CF910895CDB7DEB7E0970FB6F894DEBF6C
:1049D0000FBECDBF85B7806885BF85B7806885BFAE
:1049E00084B7877F84BF0FB6F894A8958091600044
:1049F000886180936000109260000FBE80E890E0B4
:104A00000FB6F89480936100909361000FBE81E02F
:104A10008093030180E896E09093B1018093B00108
:104A20000E94120D0E94550D86E0E4E1F1E0DE01E6
:104A3000119601900D928A95E1F7FE0131969E0143
:104A4000295F3F4FEFA7F8AB41E050E08191A82FDD
:104A5000A295AF70B0E091966C9191978F708A019A
:104A600002C0000F111F8A95E2F7C801962F982BFC
:104A700091969C93919792969C9192978095892379
:104A800092968C93E217F30709F70E941A090E9485
:104A900077098091E20084608093E20078948091AD
:104AA0006F03811599F08091E9001091EC008F70EF
:104AB000179511271795182B1092E9008091E8009F
:104AC00083FD0E94E2121F701093E90082E084BD12
:104AD00093E095BD9DE797BD80936E000E94F90C11
:104AE000811102C00E94220EEAE5F3E088E0DF01B6
:104AF0001D928A95E9F78098889884988C981092EE
:104B00004F0310924D0310924E038FEF93E090935A
:104B1000C6028093C5021092C4021092C302109282
:104B2000C2021092C10210924402109243021092EB
:104B30004202109241021092570310925603909332
:104B40004C0380934B0310924A0310924903109236
:104B50004803109247031092CA021092C9021092A1
:104B6000C8021092C702109255031092540310927B
:104B70005303109252031092510310925003A3E377
:104B8000B1E02BE331E041E050E08D918F3FA1F0A7
:104B9000E82FE295EF70F0E061A18F708A0102C00A
:104BA000000F111F8A95E2F7C801902F9095962368
:104BB00091A392A1892B82A32A173B0731F7109268
:104BC0006C0310923C0280E090E00E948530833EAE
:104BD0009E4F21F40E94F90C81111DC063EE7EEFFF
:104BE00080E090E00E94B33060E082E090E00E94BC
:104BF000993081E08093080561E083E090E00E94B5
:104C0000993060E074E184E090E00E94B3300E944B
:104C1000220E0E94F00982E090E00E94783080939A
:104C20003F0284E090E00E94853090930B058093D2
:104C30000A057CDE8FE59AEE0197F1F700C00000CF
:104C400075DE80916C0383FF08C06FEF7FEF80E01B
:104C500090E00E94B3300E94050A83E090E00E9439
:104C600078300E94D6030E94BA0E8FE090E00E9436
:104C7000803060930C0570930D0580930E05909322
:104C80000F05653010F00E94F009E0910C05F0E08E
:104C9000EE0FFF1FE955FE4F808191810E94AA0E01
:104CA00084E091E0909377038093760392E0292E3D
:104CB0003324339480916F03853049F480916F03DE
:104CC000853009F4DDC00E94A8120E949A072EDEEA
:104CD00080914002E0906C038E1153C6A1DD80915B
:104CE0001001811511F100910605109107050115BC
:104CF0001105D9F00E94BD0F801B910B20919904E2
:104D000030919A042817390780F490919C0480917F
:104D10009B04981709F400C1A8DA10929A04109223
:104D20009904109207051092060580914904811597
:104D300069F00E94BD0F20914A0430914B04821B00
:104D4000930B8F3F9F4710F40E943A1080916203AB
:104D5000811551F01092620380915C0380935D0392
:104D600080915A0380935B0380EFDCD72C0184EFA2
:104D7000D9D73C0180915703811521F080915603CA
:104D800081112BC026E533E03F932F9367E573E055
:104D90007F936F93A1E48A2EA2E09A2EB3E4AB2E08
:104DA000B2E0BB2E15E4C12E12E0D12E03E8E02EB6
:104DB00002E0F02E01EC12E022EC32E043EC52E093
:104DC00065EC72E0C2010E948C02909353038093C1
:104DD00052030F900F900F900F9080915503811503
:104DE00021F08091540381112BC0A4E5B3E0BF935F
:104DF000AF9305E513E01F930F9367EC862E62E0F7
:104E0000962E79ECA72E72E0B72EEBECCE2EE2E0D8
:104E1000DE2EF9E0EF2EF3E0FF2E07E413E028E4A6
:104E200033E049E453E06BE473E0C3010E948C0279
:104E300090935103809350030F900F900F900F9019
:104E4000409152035091530380915003909151032C
:104E500020914F03211175C04416550608F064C017
:104E60006816790608F47DC083E080934F03809133
:104E70004E03811509F475C010924E0311E072C003
:104E800080916F03843031F10E94E70A10923D0255
:104E9000A8E1B0E0E0E40FB6F894A895A093600014
:104EA0000FBEE093600083B7817F846083BF83B7C8
:104EB000816083BF7894889583B78E7F83BF0FB658
:104EC000F894A895809160008861809360001092AA
:104ED00060000FBE2BDD80916C03811509F4EECECE
:104EE00080913E02811509F4E9CE19BCF2E0F9BDCA
:104EF00009B400FEFDCF8091D8008F7D8093D8004B
:104F00008091E00082608093E0008091E00081FD6C
:104F1000FCCF0E94A812D2CE62D91092070510923F
:104F200006050E94BD0601CF68167906D0F43092BE
:104F30004F0380914D038115A1F010924D031FEF97
:104F400011C0213009F079C04416550608F46EC02E
:104F50006816790630F010924F0320934E0310929A
:104F60004D0310E0E0904704F09048040E94BD0F0C
:104F70008E199F0984369105B0F1E0905803F090A6
:104F800059030E94BD0F8E199F09059760F180910A
:104F90004604811128C0111531F180915C0390E025
:104FA0009C012F5F3F4F2370332740915D034217D1
:104FB000130699F0865A9C4F41E0113009F040E009
:104FC000479544274795DC0114964C9320935C0346
:104FD00080915A038F5F80935A030E94BD0F909374
:104FE00059038093580380E01AED20915D0390915E
:104FF0005C03921709F458C030E0F901E25AFC4F03
:10500000808187FB882780F92F5F3F4F23703327EC
:1050100020935D0390915B039F5F90935B03B12F9F
:10502000B81B8B2F0E94011281E0DFCF6816790632
:1050300008F097CF20924F0390CF223001F544160D
:10504000550670F06816790608F08BCF30924F0342
:1050500080914D03811509F484CF10924D030ECF3A
:105060006816790608F47DCF83E080934F03809122
:105070004E03811509F475CF10924E0360CF44168C
:10508000550658F06816790608F46BCF10924F0356
:1050900030924D0310924E0364CF6816790608F0E3
:1050A00060CF20924F03F4CF81110E9464080E94C8
:1050B000E70A81110E94640886E0E9EDF3E0AFA5FC
:1050C000B8A901900D928A95E1F71092DB03109236
:1050D000DC031092DD031092DE038B819C81892B0F
:1050E000811509F443C000916503109166030E9485
:1050F000BD0F9C01201B310B9091D703911509F432
:105100003BC42531310590F19F3F19F09F5F90938B
:10511000D7031B81111559F00E942F0791E011163A
:105120000CF09FEF899F802D11248093DB031C815D
:10513000111559F00E942F0791E011160CF09FEF06
:10514000899F802D11248093DC038091DB038115DE
:1051500069F01091DC03111549F00E94210780933A
:10516000DB03812F0E9421078093DC038D819E81C8
:10517000892B811509F443C00091630310916403E6
:105180000E94BD0F9C01201B310B9091D6039115FD
:1051900009F4EDC32135310590F19F3F19F09F5F70
:1051A0009093D6031D81111559F00E944F0791E08D
:1051B00011160CF09FEF899F802D11248093DD0341
:1051C0001E81111559F00E944F0791E011160CF045
:1051D0009FEF899F802D11248093DE038091DD0352
:1051E000811569F01091DE03111549F00E94210725
:1051F0008093DD03812F0E9421078093DE036FA53A
:1052000078A989ED93E00E94340881110CC0809147
:10521000DB039091DC03892B9091DD03892B909126
:10522000DE03892B81110E946E1086E0EFA5F8A99C
:10523000A9EDB3E001900D928A95E1F70E949A07DB
:1052400090916703891721F0809367030E94640897
:1052500080916F03843009F02DCD83E08093E900C5
:105260008091E80082FF26CD8091E80090E085FFE4
:1052700005C00E94E908811529F191E08091E800BC
:105280008B778093E800911509F414CD0091720397
:1052900010917303E9810115110581F1EE3F09F0C9
:1052A0004FC08A81833020F08550833008F048C099
:1052B000EA81EE3008F044C0F0E0E755FD4CCE0145
:1052C0000196CCC600E210E0FE0131967F0180918C
:1052D000E80085FD0AC08091E8008B778093E800A4
:1052E0000E94E908811599F3C8CF8091F100D70198
:1052F0008D937D010150104051F7BFCFE43148F448
:10530000E11549F0E150E33130F4F0E0E954FD4CAF
:10531000A5C6EE3F69F28FEF898312C01A8289E039
:105320008B830EC08A81823081F08330B1F081306E
:1053300091F70E946408A8D66B837C838D839E833B
:10534000CE0101960E943909B5CC88E290E0D0D612
:105350001B821C821D828E83F3CF80916D039091FE
:105360006E03892B69F380916C03DACF8A818230D6
:1053700091F66B817C818D819E8186D688E290E05A
:10538000D8D6DECF4C816B818A810E941C0C982775
:10539000892798279E838D83D3CF2D813E81322705
:1053A000232732274C816B818A810E94A10AC8CFB2
:1053B0000E94910DC5CF80E18A83C2CF83E08A83AA
:1053C00087E0AECF8C818D3108F0BACF8A809B8088
:1053D000982489249824A12CB12C8E010F5F1F4F93
:1053E0007801E80EF11C0E151F0509F4A9CF80E025
:1053F000B7E08B16B3E09B06A104B10420F4C4010E
:1054000087509F4F75D6F80184830F5F1F4FFFEFC2
:105410008F1A9F0AAF0ABF0AE6CF80916D03909161
:105420006E03892B09F48CCF8C818D3108F088CFE5
:10543000882E912CA12CB12CCA80DB80DC24CD24B9
:10544000DC24E12CF12C8E010F5F1F4F412C512CDD
:105450003201481459046A047B0408F071CF27E034
:10546000C21623E0D206E104F10438F4D801149600
:105470006C91C60187509F4F5CD6BFEF4B1A5B0AF9
:105480006B0A7B0AEFEFCE1ADE0AEE0AFE0A0F5F06
:105490001F4FDFCF0E94E80D53CF84E08DCF8C816A
:1054A0008D3108F04DCF882E912CA12CB12CCA80C3
:1054B000DB80DC24CD24DC24E12CF12C412C512C8C
:1054C00032018E010B5F1F4F481459046A047B049C
:1054D00008F036CF80E0F0E4CF16D104E104F10407
:1054E00018F4C601899604D6D8018D938D01BFEFBB
:1054F0004B1A5B0A6B0A7B0AEFEFCE1ADE0AEE0A42
:10550000FE0AE2CF2C81622E712C2D3108F018CFCB
:105510008A819B819827892798274C01A12CB12C3F
:105520008034910508F00CCF422F50E060E070E02D
:105530004BA75CA76DA77EA740E450E060E070E059
:10554000481959096A097B09421751056105710516
:1055500008F4F6CE20916D0330916E03232B09F0F1
:105560003EC07C0159E2E50EF11C80FBCC24DD2419
:10557000C0F880FF0BC08896BBD59D8189279827EE
:10558000892781159C4711F48FEF8D838BA59CA5EE
:10559000ADA5BEA5880D991DAA1DBB1D80FF17C016
:1055A00083010150110955E0452E512C4C0E5D1E12
:1055B000400E511EC701860D971D9AD5D2019C91B0
:1055C00081159C4719F48FEFF20180833801FE01A9
:1055D0003196EC0DFD1D2FEFC614D70438F08E0167
:1055E0000F5F1F4FC12CD12C760124C0948185817F
:1055F00081159C4711F42483258312E0C10ED11C30
:105600003296EACF20E482169104A104B10430F46A
:10561000D80114966C91C40189968BD5BFEFCB1A33
:10562000DB0AEB0AFB0AEFEF8E1A9E0AAE0ABE0AED
:105630000F5F1F4F2BA53CA54DA55EA5C216D30637
:10564000E406F506F8F27CCE80916D0390916E032E
:10565000892B09F475CECE0101960E9439093FEFDE
:1056600040E752E0315040405040E1F700C00000B8
:10567000F2CA88E0EBE1F1E0DE01919601900D9233
:105680008A95E1F7FE0132968FE1DF011D928A953E
:10569000E9F786E0898388E07F96DE011596019020
:1056A0000D928A95E1F74CCE8CE7898381E08A835D
:1056B0001B821C8245CE0B811C81012E000C220B0B
:1056C000330B45E0000F111F221F331F4A95D1F7FE
:1056D000B901A801405E5F4F6F4F7F4F40175107E0
:1056E0006207730708F42CCE0C37B1E01B072105C5
:1056F000310508F025CE4D37E1E05E076105710503
:1057000020F04CE751E060E070E0401B510BB80125
:1057100066507D4FC0D414CE4AE150E06FEF70E088
:10572000CE010796CED480916D0389830A831B82B4
:1057300084E08C831D8285E00ECE81E090E0909322
:1057400073038093720382E390E090936B038093E2
:105750006A030E94BD0F9093690380936803F0CDA4
:105760000115110571F1D0906C03E0906803F09081
:1057700069030E94BD0F8E199F098536910540F17E
:10578000D5FE26C0D4FE24C00E94BD0F90936903AD
:105790008093680380916A0390916B0301979093C3
:1057A0006B0380936A03892B61F410927303109248
:1057B000720381E090E090936E0380936D0300E0AC
:1057C00010E080916D0389830A8380916A03A8CDDC
:1057D00082E390E090936B0380936A03F2CF109280
:1057E0006E0310926D03ACCD40E250E06FEF70E0BD
:1057F00068D4A6CD2B81243009F473C010F521158F
:1058000009F462C0233009F09BCD2C816AE0CE01FF
:105810008196FC01062F11920A95E9F7283008F0CD
:105820005EC0629FB001112467587F4F4AE050E08C
:105830004FD480E089838AE0FE01B196DE011296A2
:105840002ECF273009F47AC0283009F079CD6C8149
:1058500086E0FE013596DE01919601900D928A95C3
:10586000E1F789A19AA18115FCE79F0741F42091F6
:105870006D0330916E03232B11F480E090E09AA326
:1058800089A38BA19CA181150CE7900741F420917D
:105890006D0330916E03232B11F480E090E09CA304
:1058A0008BA38FEF683060F416E0619FB001112484
:1058B00067537F4F46E050E0CE01819658D480E098
:1058C00089830E94550D3CCD2FE1DC011D922A9564
:1058D000E9F788E08A838C8383E088A331CD8FEF5A
:1058E000A9CF6C818AE0FE013596DE019196019088
:1058F0000D928A95E1F789A59AA581151CE7910774
:1059000041F420916D0330916E03232B11F480E05C
:1059100090E09AA789A78FEF683060F42AE0629F31
:10592000B001112467587F4F4AE050E0CE018196C4
:105930001ED480E089830E94120D02CD2C8166E086
:10594000CE018196DC01E62F1D92EA95E9F7283019
:1059500060F4629FB001112467537F4F46E050E02E
:10596000B7D380E0898386E067CF8FEFFBCF2B3002
:10597000310508F014CC43CC2B30310508F0C6CBF0
:10598000F5CBF82EFE2400E011E08F2D8123811548
:10599000A9F009831A820E94BD0F9C838B833D82EC
:1059A00091E08E2D8123811101C090E09E83498179
:1059B0005A816B817C818D810E94E2210F5F110FE2
:1059C000083019F7E09240020E94640888C9789470
:1059D0001F921FB61F9211248F939F93AF93BF9373
:1059E0008091D2019091D301A091D401B091D501C1
:1059F0000196A11DB11D8093D2019093D301A09374
:105A0000D401B093D501BF91AF919F918F911F9019
:105A10001FBE1F9018951F920F920FB60F92112460
:105A20002F933F934F935F936F937F938F939F93A6
:105A3000AF93BF93EF93FF938091E10082FF09C082
:105A40008091E20082FF05C08091E1008B7F80930E
:105A5000E1008091DA0080FF23C08091D80080FFB0
:105A60001FC08091DA008E7F8093DA008091D90088
:105A700019BC80FFA6C082E089BD09B400FEFDCF3D
:105A800081E080936F038091C101811109C00E9460
:105A90001A090E9477098091E20084608093E200F5
:105AA0008091E10080FF1AC08091E20080FF16C063
:105AB0008091E2008E7F8093E2008091E20080611D
:105AC0008093E2008091D80080628093D80019BC56
:105AD00085E080936F0383E0809303018091E10070
:105AE00084FF2EC08091E20084FF2AC019BC82E0AE
:105AF00089BD09B400FEFDCF8091D8008F7D8093D1
:105B0000D8008091E1008F7E8093E1008091E200D7
:105B10008F7E8093E2008091E20081608093E200BA
:105B20008091C001811509F451C084E080936F0316
:105B300080916F03843009F051C082E080930301AB
:105B40008091E10083FF2CC08091E20083FF28C098
:105B50008091E100877F8093E10082E080936F0372
:105B60001092C0018091E1008E7F8093E1008091CE
:105B7000E2008E7F8093E2008091E200806180935A
:105B8000E20042E060E080E00E9447098091F0007E
:105B900088608093F00081E080930301809302018C
:105BA000FF91EF91BF91AF919F918F917F916F91F5
:105BB0005F914F913F912F910F900FBE0F901F90CB
:105BC000189510926F031092C1016ACF8091E30083
:105BD00087FF02C083E0AACF81E0A8CF81E0AECFEB
:105BE0001F920F920FB60F921124EF92FF920F9314
:105BF0001F932F933F934F935F936F937F938F9355
:105C00009F93AF93BF93CF93EF93FF9309EE10E071
:105C1000F8018081C091EC008F70C795CC27C795A3
:105C2000C82B108280EFE82EF12CF7018081877F4E
:105C3000808378940E94E212F8011082F70180813B
:105C400088608083CF70F801C083FF91EF91CF917E
:105C5000BF91AF919F918F917F916F915F914F9184
:105C60003F912F911F910F91FF90EF900F900FBEDA
:105C70000F901F901895803F09F188F4843901F145
:105C800040F48533F9F08633F9F0843339F583E253
:105C900008958639D9F0873909F582E20895853F5C
:105CA000B9F030F4813FB1F0843FC1F484E008954D
:105CB000863F91F0873F91F487E0089580E0089552
:105CC00080E2089584E2089585E2089581E20895CE
:105CD00085E0089581E0089586E008958FE10895B4
:105CE00095E890937A00982F9072906890937B003B
:105CF0008F7190911101892B80937C0080917A00A3
:105D0000806480937A0080917A0086FDFCCF809138
:105D100078002091790090917A009F7790937A0093
:105D2000922F0895A8DFDCCF289A219A229A2398EF
:105D30002B9880E58CBD0895FC01809113018F3F65
:105D400009F085C080818F3F09F481C01092110550
:105D50008181811519F080E28093110592818091F3
:105D60001105923009F44FC0933009F450C084609B
:105D7000913009F449C08381948121E030E02817F3
:105D8000390708F446C0809111052032310509F425
:105D900056C008F041C02830310509F44BC020310D
:105DA000310509F44AC02230310509F43FC08CB5F1
:105DB00090911105892B8CBD80911005811519F0EA
:105DC0008DB581608DBD2081209313014581409365
:105DD0001201E22FE295EF70A1E2AE0FB0E03C912C
:105DE0002F7081E090E001C0880F2A95EAF7232FF9
:105DF000282B2C93EE5DF0E09081411125C0892B7A
:105E0000808381E00895886080931105B4CF8C6011
:105E1000FBCF220F331FB3CF2034310599F08360BD
:105E20002038310521F680931105C1CF81E08093A0
:105E30001005BDCF91E0909310058160F4CF91E003
:105E4000909310058260EFCF80958923D9CF80E0B1
:105E50000895A6E0B0E0EEE2FFE2B2C089836A8373
:105E60004B833D832C8381E08E83CE01019664DFDA
:105E70002696E2E0C1C0CF93DF938EBD0E94BD0F96
:105E8000EC010DB407FE05C08EB590E0DF91CF9117
:105E900008950E94BD0F8C1B9D0B8436910588F3DD
:105EA0008EEF9FEFF3CFCF93DF931EBC0E94BD0F09
:105EB000EC010DB407FE05C08EB590E0DF91CF91E7
:105EC00008950E94BD0F8C1B9D0B8436910588F3AD
:105ED0008EEF9FEFF3CF0F931F93CF93DF93EC01E0
:105EE0008C01060F171FC017D10739F480E090E02E
:105EF000DF91CF911F910F9108958991BCDF97FF9A
:105F0000F2CF8EEF9FEFF4CF0F931F93CF93DF93DA
:105F1000EC018C01060F171FC017D10739F480E080
:105F200090E0DF91CF911F910F910895BCDF97FD15
:105F300002C08993F1CF8EEF9FEFF3CF2091130131
:105F40002F3F51F1E22FE295EF70A1E2AE0FB0E0EA
:105F50003C912F7081E090E001C0880F2A95EAF70C
:105F6000232F282B2C93EE5DF0E0209112019081DD
:105F7000211599F0892B80838FEF809313018DB5C4
:105F80008E7F8DBD9CB580911105809589238CBD38
:105F90001092110510921005089580958923EBCF7A
:105FA0002F923F924F925F926F927F928F929F9229
:105FB000AF92BF92CF92DF92EF92FF920F931F9317
:105FC000CF93DF93CDB7DEB7CA1BDB0B0FB6F894C8
:105FD000DEBF0FBECDBF09942A88398848885F8408
:105FE0006E847D848C849B84AA84B984C884DF8079
:105FF000EE80FD800C811B81AA81B981CE0FD11D5D
:106000000FB6F894DEBF0FBECDBFED010895AA1BF9
:10601000BB1B51E107C0AA1FBB1FA617B70710F093
:10602000A61BB70B881F991F5A95A9F780959095C5
:10603000BC01CD01089597FB072E16F4009406D0FD
:1060400077FD08D0E4DF07FC05D03EF490958195FC
:106050009F4F0895709561957F4F0895EE0FFF1F34
:106060000590F491E02D0994082E81700694069411
:10607000811D0694811D0694811D0694811D069440
:10608000811D0694801D0895692796276927782722
:10609000872778270895FB01DC0102C005900D9247
:1060A00041505040D8F70895FB01DC0104C08D91A8
:1060B0000190801921F441505040C8F7881B990B7A
:1060C0000895DC0101C06D9341505040E0F7089500
:1060D000DC01CB01FC01F999FECF06C0F2BDE1BDA8
:1060E000F89A319600B40D9241505040B8F7089597
:1060F000F999FECF92BD81BDF89A992780B5089590
:10610000A6E1B0E044E050E0E5CFA8E1B0E042E035
:1061100050E0E0CFDC01A40FB51F4150504040F0EB
:10612000CB01840F951F2E9105D041505040D8F7D8
:106130000895262FF999FECF92BD81BDF89A019757
:1061400000B4021639F01FBA20BD0FB6F894FA9ABF
:10615000F99A0FBE08950396272FECDFEADF252F6B
:10616000E9DF242FE7CF0196272FE4DFE2CFDC0120
:10617000CB0102C02D9105D041505040D8F7089571
:10618000262FF999FECF1FBA92BD81BD20BD0FB653
:10619000F894FA9AF99A0FBE019608955058BB27C1
:1061A000AA270ED0E5C0D6D030F0DBD020F031F4F5
:1061B0009F3F11F41EF4CBC00EF4E095E7FBC1C085
:1061C000E92FE7D080F3BA176207730784079507B2
:1061D00018F071F49EF5FFC00EF4E0950B2EBA2F67
:1061E000A02D0B01B90190010C01CA01A0011124DD
:1061F000FF27591B99F0593F50F4503E68F11A1689
:10620000F040A22F232F342F4427585FF3CF469519
:1062100037952795A795F0405395C9F77EF41F163B
:10622000BA0B620B730B840BBAF09150A1F0FF0F05
:10623000BB1F661F771F881FC2F70EC0BA0F621FF1
:10624000731F841F48F4879577956795B795F795E1
:106250009E3F08F0B3CF9395880F08F09927EE0F73
:1062600097958795089504D06894B111B5C00895A5
:1062700098D088F09F5790F0B92F9927B751A0F088
:10628000D1F0660F771F881F991F1AF0BA95C9F7CA
:1062900012C0B13081F09FD0B1E008959CC0672F4B
:1062A000782F8827B85F39F0B93FCCF3869577957A
:1062B0006795B395D9F73EF4909580957095619563
:1062C0007F4F8F4F9F4F0895E89409C097FB3EF48E
:1062D00090958095709561957F4F8F4F9F4F992333
:1062E000A9F0F92F96E9BB279395F69587957795B1
:1062F0006795B795F111F8CFFAF4BB0F11F460FF71
:106300001BC06F5F7F4F8F4F9F4F16C0882311F0C8
:1063100096E911C0772321F09EE8872F762F05C0DC
:10632000662371F096E8862F70E060E02AF09A9577
:10633000660F771F881FDAF7880F9695879597F96C
:10634000089597F99F6780E870E060E008959FEFF7
:1063500080EC089500240A941616170618060906FC
:10636000089500240A9412161306140605060895CB
:10637000092E0394000C11F4882352F0BB0F40F453
:10638000BF2B11F460FF04C06F5F7F4F8F4F9F4F93
:10639000089557FD9058440F551F59F05F3F71F015
:1063A0004795880F97FB991F61F09F3F79F087957C
:1063B0000895121613061406551FF2CF4695F1DF05
:1063C00008C0161617061806991FF1CF8695710595
:1063D000610508940895E894BB2766277727CB01C9
:1063E00097F908950BD0C4CFB5DF28F0BADF18F0C5
:1063F000952309F0A6CFABCF1124EECFCADFA0F3CF
:10640000959FD1F3950F50E0551F629FF001729F49
:10641000BB27F00DB11D639FAA27F00DB11DAA1F68
:10642000649F6627B00DA11D661F829F2227B00DB5
:10643000A11D621F739FB00DA11D621F839FA00D40
:10644000611D221F749F3327A00D611D231F849F90
:10645000600D211D822F762F6A2F11249F575040E7
:106460008AF0E1F088234AF0EE0FFF1FBB1F661F82
:10647000771F881F91505040A9F79E3F510570F03B
:1064800060CFAACF5F3FECF3983EDCF3869577951B
:106490006795B795F795E7959F5FC1F7FE2B880F36
:1064A000911D9695879597F90895F894FFCF9510CB
:1064B0009B109E10A410B910B910B910B910B910E2
:1064C000B910B910B910A710AC10B010B610DB108D
:1064D000E110E510C313E913EF13E913EF134214AE
:1064E0006414EF136B157815A81A101BB01A7B1AD9
:1064F0007F1AB41A831AB81AC41A8F1A091B931A6E
:10650000C81A971ACC1AF11A9B1AD01AF81AA01A9C
:10651000D61ADE1A871ABC1A8B1AC01AA41ADA1AEB
:10652000E81A011B071B751AAC1A171B531A571AC6
:106530004A1A4F1A5B1A5F1A631A7F1C7F1CB91C18
:10654000B91C6E1D891DE11CE11C8E1D031E151E4C
:10655000151E392B542B5B2BA029A0298C2B9D2B8E
:10656000B02BEF2BF42BA029A029A029FA2B8E29E0
:106570009229B629C229CD29D8298B298B298B2983
:106580008B29242BDB29DE29E2290D2A4A2A4D2AD0
:046590004F2A822AE2
:106594000000010061086B0A7008810A860A620A19
:1065A400014001FF3496F1F5F6F700841C3408C964
:1065B400C5B4370044227B49012701AC004F02686F
:1065C4000288029492C63697666737E200E900EAC9
:1065D40000B500B600B700CD008301CC008A01925B
:1065E4000194012102230224022502260227022A01
:1065F40002B300B4006F0070009F01CB019F02A0A2
:1066040002E200E900EA00B500B600B700CD00835D
:1066140001CC008A01920194012102230224022563
:1066240002260227022A02B300B4006F0070009F02
:1066340001CB019F02A0022003B0044006600900C0
:00000001FF
